S123A100FFB3F3BDA7C0FFB3F5A60026037EA275BDA98B7FB3EDCE0000FFB505FFB3EEFE32
S123A120B5016F00FFB503FEB3F5BDA9D227037EA272CE0000FFB4FF7FB50F7FB5077FB573
S123A14008BDAA5C24037EA1A3BDA5E77DB4F92714FEB4F9BDA6592506BDA28E7EA272FE8A
S123A160B4F9BDA6227DB4FB271CFEB4FBBDA6ACBDA6F52406BDA27E7EA272BDA3BE240645
S123A180BDA27E7EA272FEB505F6B50F3AFFB505FCB505F3B507FDB505FEB4FF08FFB4FF60
S123A1A07EA13881002706CEB138BDA780FEB3F5BDA7C0A600270A812D2706FFB3F57EA1B9
S123A1C027FEB3F3BDA7C0FFB3F57CB3EDCE0000FFB505FFB3EEFEB3F5BDA9D227037EA27A
S123A1E072CE0000FFB4FF7FB50F7FB5077FB508BDAA5C24037EA249BDA5E77DB4FB271CA4
S123A200FEB4FBBDA6ACBDA6F52406BDA27E7EA272BDA3BE2406BDA27E7EA2727DB50F276E
S123A22003BDA9707DB3F02703BDA30FFEB505F6B50F3AFFB505FCB505F3B507FDB505FE09
S123A240B4FF08FFB4FF7EA1E781002706CEB138BDA780FEB3F5BDA7C0A600270A812D27C8
S123A26006FFB3F57EA1D67DB3F02703BDA68FBDA2DE7ED003CEAFFCBDA7807EA2727DB34F
S123A280F12653BDA2FDCEB161BDA78020487DB3F12643BDA2FDCEB173BDA78020387DB384
S123A2A0F12633BDA2FDCEB185BDA78020287DB3ED27237DB3F1261EBDA2FDCEB197BDA722
S123A2C08020137DB3ED270E7DB3F12609BDA2FDCEB1ACBDA780FEB3EE08FFB3EE39FEB389
S123A2E0EE2713CEB10DBDA780CEB3EEBDA7B4BDA78BBDA78B39CEB118BDA78039FEB3F5CA
S123A300BDA76E863ABD7FE8CEB4FFBDA7B439CEB4FFBDA7B4CEB505BDA7B47FB3E0BDA306
S123A3205DBDA7B8BDA7B8CEB3F7BDA780BDA78BB6B50FB1B3E02724BDA7B8BDA7B8BDA794
S123A340B8BDA7B8BDA7B8BDA7B8BDA7B8BDA7B8BDA7B8BDA7B8BDA384BDA78B395FCEB58F
S123A36010F1B50F270DC1042719BDA7B65CF7B3E020EEC104270CBDA7B8BDA7B8BDA7B881
S123A3805C20F039F6B3E0CEB5103AF1B50F270ABDA7B65CC503270320F139BDA78BBDA7D3
S123A3A0B8BDA7B8BDA7B8BDA7B8BDA7B8BDA7B8BDA7B8BDA7B8BDA7B8BDA7B820CD7FB5C4
S123A3C00FFEB50DA6092A037EA4EE810527458104274DFEB4FDA600812326037EA44D81C1
S123A3E02C26037EA483A601812C26037EA483A602812C26037EA483A603812C26037EA479
S123A40083FEB4FDA600813C27037EA4A808FFB4FD7EA4CAA608B7B5108601B7B50F0C399A
S123A420A604B7B5108602B7B50FFEB4FDBDA7DF24037EA5E2FCB3EBB3B505830002F7B599
S123A440114D270781FF2703BDA2C30C39FEB50DA60426037EA4ECB7B510A6094CB7B50FC8
S123A460FEB4FD08BDA7DF24037EA5E2B6B50F81022708FEB3EBFFB5110C39B6B3ECB7B51F
S123A480110C39FEB50DA6062762B7B5108602B7B50FFEB4FDBDA7DFB6B3ECB7B5117DB3FA
S123A4A0EB2703BDA2AE0C39FEB50DA607273DB7B5108603B7B50FFEB4FDBDA7DF24037E49
S123A4C0A5E2FEB3EBFFB5110C39FEB50DA605271BB7B5108602B7B50FFEB4FDBDA7DF2409
S123A4E0037EA5E2B6B3ECB7B5110C390D39818026037EA521818426037EA53481852603D1
S123A5007EA547818126037EA56B818226037EA591818326037EA5BA818626037EA5E00DEA
S123A52039FEB4FDBDA7DF24037EA5E2FEB3EBFFB5050C39FEB4FDBDA7DF24037EA5E2FC0C
S123A540B3EBFDB5070C39FEB4FDBDA7DF24037EA5E2FEB4F9BDA65924037EA29EFEB3E45C
S123A560BDA7C008FCB3EBED000C39FEB4FDBDA7DF24037EA5E2B6B3ECCEB510F6B50F3AE5
S123A580A7007CB50FFEB3E9A60008812C27DF0C39FEB4FDBDA7DF24037EA5E2CEB510F6E9
S123A5A0B50F3AFCB3EBED007CB50F7CB50FFEB3E9A60008812C27DC0C39FEB4FDA600B749
S123A5C0B3E008A6002717B1B3E027123CCEB510F6B50F3AA7007CB50F38270220E40C3927
S123A5E00C39BDA2AE0C39CE0000FFB4F9FFB4FBFFB4FDCEB3F7A6002727812A2723813BCB
S123A600271F8120270781092703FFB4F9BDA7C06D00270DFFB4FBBDA7C06D002703FFB4E0
S123A620FD39A600BDA95B251EA600271A8120271681092712813A270E3CFEB503A700081D
S123A640FFB503380820E2FEB5036F00FCB505ED010808086F00FFB503FFB3E2FEB501FFAF
S123A660B3E46D002721BDA70D240EFEB3E4BDA7C0080808FFB3E420E9FEB3E4BDA7C008B6
S123A680EE00FFB3E60C397FB3E67FB3E70D39CEB101BDA780FEB5016D00270FBDA78008CD
S123A6A0BDA7B8BDA7B4BDA78B20ED39A60084DFB7B509A60184DFB7B50AA60284DFB7B5B8
S123A6C00BA6038140230A817A220684DFB7B50C39862020F8A600B1B5092617A601B1B580
S123A6E00A2610A602B1B50B2609A603B1B50C26020C390D39C60ACEAA8D6D00270DBDA627
S123A700D524033A20F4FFB50D0C390D39FEB3E23CFEB3E43CFEB3E4A6008D30271B3CFE8B
S123A720B3E2E60008FFB3E2381126030820E938FFB3E438FFB3E20D39FEB3E2A6008D0CC9
S123A74026ED38FFB3E438FFB3E20C394D271D812027198109271581202711813A270D8182
S123A7602C2709812B2705812D2701394F39A60027188120271481092710BD7FE80820EE4E
S123A780A6002706BD7FE80820F63936860DBD7FE8860ABD7FE8323944444444840F8B30FD
S123A7A0813923028B277E7FE8A600BDA798A600087EA79C8DF38DF1368620BD7FE83239A5
S123A7C0A600271781202707810927030820F1A60027088120270581092701390820F07FD1
S123A7E0B3EB7FB3EC862BB7B3E8A600812B2606B7B3E8082008812D2604B7B3E808FFB3B2
S123A800E9A600812427298125272F81272730812A2737BDA95B251D7DB3ED270ABDA6599F
S123A8202403BDA29E202C7FB3EB7FB3EC0C2023BDA89D201EBDA8CD2019BDA910201408BD
S123A840A600B7B3EC7FB3EB2038FCB505FDB3E60C20002532B6B3E8812D2608FCB3EBB33A
S123A860B3E62006FCB3EBF3B3E6FDB3EBBDA88CA600270E812B26037EA7E5812D26037E54
S123A880A7E5FFB3E90C39FFB3E90D39FEB3E9A600BDA74C27030820F6FFB3E9397FB3E643
S123A8A07FB3E7A6008124260108A600BDA74C2718BDA9412415FDB3E0FCB3E60505050553
S123A8C0FAB3E0FDB3E60820E10C390D397FB3E67FB3E7A600BDA74C271EBDA941241B818A
S123A8E0092E17BDA8FC7FB3E0B7B3E1FCB3E6F3B3E0FDB3E60820DB0C390D393637FCB3ED
S123A900E605FDB3E00505F3B3E0FDB3E63332397FB3E67FB3E7A6008125260108A600BDE5
S123A920A74C2719BDA94124D181012E12B7B3E0FCB3E605FAB3E0FDB3E60820E00C390D21
S123A94039271680302B1281092F0C84DF81112D0881162E0480070D390C3936815F270A7F
S123A96084DF81402307815A2E03320C39320D397DB3F227155FF1B50F270FCEB5103AA66F
S123A98000FEB5053AA7005C20EC39CE0100FFB501FEB3F3A600272C812D2705BDA7C0203A
S123A9A0F308A60084DF814C26037CB3F0814526037CB3F1814426037CB3F281542603BDA1
S123A9C0A9C520D83908BDA89D25F9FCB3E6FDB50139FFB1C4FFB1D6CEB1C2BDD0067DB12F
S123A9E0C32615B6B1C685402618CE0000FFB1DCFFB1DEFFB1DA4F39CEB127BDA780B6B13A
S123AA00C339CEB14ABDA78086FF39FEB1DCBCB1C92246FEB1DEBCB1CB273E188401188C37
S123AA2000002612CEB1D4BDD0067DB1D5262BFEB1DA08FFB1DAFCB1DE8401C3B1E018A663
S123AA400018FCB1DEC30001FDB1DE2409FCB1DCC30001FDB1DC180C394F0D39CEB3F7FF92
S123AA60B4F7BDAA0B251F810A2714810D27F3FEB4F7A700088CB4F62205FFB4F720E3FEA3
S123AA80B4F76F000C39FEB4F76F000D39414444418B9BABBB000141444442CBDBEBFB00C7
S123AAA00141444444C3D3E3F3000241424120000000001B05414443418999A9B900014143
S123AAC0444342C9D9E9F90001414E44418494A4B40001414E4442C4D4E4F400014249543A
S123AAE0418595A5B5000142495442C5D5E5F50001434C522000006F7F0000434C524100F5
S123AB000000004F05434C5242000000005F05434D50418191A1B10001434D5042C1D1E13B
S123AB20F1000143424120000000001105434F4D20000063730000434F4D410000000043EB
S123AB4005434F4D420000000053054E4547200000607000004E4547410000000040054EFB
S123AB60454742000000005005444141200000000019054445432000006A7A00004445430E
S123AB8041000000004A0544454342000000005A05454F52418898A8B80000454F5242C81D
S123ABA0D8E8F80000494E432000006C7C0000494E4341000000004C05494E43420000006F
S123ABC0005C054C4441418696A6B600014C444142C6D6E6F600014C444420CCDCECFC0075
S123ABE0024D554C20000000003D054F5241418A9AAABA00014F524142CADAEAFA00015056
S123AC005348410000000036055053484200000000370550554C4100000000320550554C56
S123AC2042000000003305524F4C20000069790000524F4C41000000004905524F4C4200FC
S123AC400000005905524F5220000066760000524F5241000000004605524F5242000000EF
S123AC6000560541534C2000006878000041534C4100000000480541534C420000000058AD
S123AC800541534C44000000000505415352200000677700004153524100000000470541E5
S123ACA05352420000000057054C5352200000647400004C5352410000000044054C5352F8
S123ACC0420000000054054C535244000000000405535441410097A7B7000053544142004F
S123ACE0D7E7F700005354442000DDEDFD0000535542418090A0B0000153554242C0D0E0A1
S123AD00F00001535542448393A3B3000253424120000000001005534243418292A2B20016
S123AD200153424342C2D2E2F2000154414220000000001605544241200000000017055412
S123AD4053542000006D7D000054535441000000004D0554535442000000005D0541494D3A
S123AD60200071610000034F494D2000716100000345494D2000756500000354494D20001E
S123AD807B6B000003435058208C9CACBC000244455820000000000905444553200000001E
S123ADA0003405494E5820000000000805494E53200000000031054C445820CEDEEEFE005A
S123ADC0024C4453208E9EAEBE00025354582000DFEFFF000053545320009FAFBF00005469
S123ADE05853200000000035055453582000000000300541425820000000003A05505348D1
S123AE0058000000003C0550554C58000000003805584744580000000018054252412020A2
S123AE20000000000442524E202100000000044243432024000000000442435320250000B6
S123AE40000004424C4F2025000000000442455120270000000004424745202C0000000087
S123AE6004424754202E000000000442484920220000000004424C45202F0000000004421A
S123AE804C5320230000000004424C54202D0000000004424D49202B0000000004424E4599
S123AEA020260000000004425643202800000000044256532029000000000442504C202ABD
S123AEC00000000004425352208D00000000044A4D502000006E7E00004A535220009DAD86
S123AEE0BD00004E4F502000000000010552544920000000003B05525453200000000039DD
S123AF000553574920000000003F0557414920000000003E05534C5020000000001A05431C
S123AF204C4320000000000C05434C4920000000000E05434C5620000000000A0553454353
S123AF4020000000000D0553454920000000000F0553455620000000000B05544150200083
S123AF600000000605545041200000000007054F524720000000000080464342200000003E
S123AF800000814644422000000000008246434320000000000083524D422000000000004E
S123AFA08445515520000000000085454E4420000000000086535043200000000000864E22
S123AFC0414D200000000000864E414D4500000000008654544C200000000000864F505405
S123AFE02000000000008650414720000000000086504147450000000000860036333031BC
S123B0002F3633303320617373656D626C65722076312E302E310D0A44616E69656C2054F7
S123B0207566766573736F6E20323031372D323031390D0A53796E7461783A2061736D2057
S123B0405B66696C65735D205B2D6C5D205B2D655D205B2D645D205B2D74585858585D0DF7
S123B0600A4F7074696F6E733A0D0A20202D6C2020202020205072696E74206C697374699A
S123B0806E670D0A20202D6520202020202048696465206572726F72730D0A20202D6420EF
S123B0A02020202020417373656D626C65206469726563746C7920746F206D656D6F727984
S123B0C00D0A20202D745858585820204D6F76652073796D626F6C207461626C6520746F5C
S123B0E02061646472657373202458585858202864656661756C74202430313030290D0A30
S123B100000D0A4C6162656C733A0D0A000D0A4572726F72733A20000D0A4E6F2065727245
S123B1206F72730D0A0A0046696C65206E6F7420666F756E640D0A0046696C65207265617A
S123B14064206572726F720D0A00456E7472792069732061206469726563746F72790D0A8B
S123B16000496E76616C6964206F702D636F64650D0A004475706C6963617465206C61623C
S123B180656C0D0A004C6162656C206E6F7420666F756E640D0A00496E76616C69642065D3
S123B1A0787072657373696F6E0D0A004272616E6368206F7574206F662072616E67650D94
S123B1C00A0001000000000000000000000000000000000011000000B1E0000000000000BE
S116B3E00000000000000000000000000000000000000056
S9030000FC
